:020000040800F2
:1000000060070020A1110008B9030008BB03000825
:10001000BF030008C3030008C70300080000000076
:10002000000000000000000000000000CB030008FA
:10003000CD03000800000000CF030008D103000832
:10004000BB110008BB110008BB110008BB11000860
:10005000BB110008BB110008BB110008BB11000850
:10006000BB110008BB110008BB110008BB11000840
:10007000BB110008BB110008BB110008BB11000830
:10008000BB110008BB110008BB110008BB11000820
:100090001B070008BB110008BB110008BB110008BA
:1000A000BB110008BB110008BB110008BB11000800
:1000B000BB110008D90C0008BB110008BB110008D7
:1000C000BB110008BB110008BB110008BB110008E0
:1000D000BB110008CB0E000861110008BB1100081D
:1000E000BB110008BB110008BB11000800F002F8AA
:1000F00000F03AF80AA090E8000C82448344AAF188
:100100000107DA4501D100F02FF8AFF2090EBAE885
:100110000F0013F0010F18BFFB1A43F0010318473B
:100120002035000040350000103A24BF78C878C15F
:10013000FAD8520724BF30C830C144BF04680C60ED
:10014000704700000023002400250026103A28BF35
:1001500078C1FBD8520728BF30C148BF0B60704739
:100160001FB51FBD10B510BD03F037FA1146FFF7DC
:10017000F7FF00F0B3F803F055FA03B4FFF7F2FF0E
:1001800003BC00F047FE000010B5002402217F48A8
:1001900001F07FFE08B944F0080404217B4801F017
:1001A00078FE08B944F004044FF48061774801F008
:1001B00070FE08B944F002044FF40061734801F086
:1001C00068FE08B944F00104204610BD10B500F0E7
:1001D00070F9482000F0E8FC00F016FE41F61F41DF
:1001E00041F2873000F032FD4FF4165000F0AAFEC5
:1001F00000F00AFC00F0A4FC00F0DCF910BD30B502
:100200000246002300BF0AE014780D78AC4201D00A
:10021000002006E00120521C491C5C1CE3B2062BA6
:10022000F2DB00BF30BD10B5584801F03BFE00F4D2
:100230007070B0F5707F50D05548007800284CD1D0
:10024000544908603C2054490870504801F02AFE87
:1002500000F470744D4801F025FE00F47070B0F5A4
:10026000E07F29D0B0F5307F1BD0B0F5507F0DD0A6
:10027000B0F5607F2BD1012045490870FF20474928
:100280000870002048708870C87021E00120404943
:100290000870FF2041494870002008708870C870BD
:1002A00016E001203A490870FF203C498870002080
:1002B00008704870C8700BE0012035490870FF20B5
:1002C0003649C870002048708870087000E000BF90
:1002D00000BF4FF47A7000F081FC10BDFFF776FF8D
:1002E000FFF752FF044604F111002D490870002069
:1002F000284908602B49C1F8B40101202A49087037
:1003000000F022FF012000F0F2FE012000F0EFFEDD
:10031000012000F0ECFE002023490870234908600A
:100320000120091D086000202149088001201F4983
:10033000091D0860091F086000200860012008608E
:100340000020086020E012480078E8B10020194938
:1003500008701649091D08600120134908700C48EF
:10036000007800F0C4FE0020094908700E490870AA
:100370000C49C1F8B00101200C49091D08600D4964
:1003800008700849C1F8B801DDE70000000C014021
:100390003C000020900121424900002088000020FC
:1003A0006B0000200080214210000020B08121421B
:1003B000460000203D000020704700BFFEE700BF60
:1003C000FEE700BFFEE700BFFEE7704770477047DB
:1003D000704700000CB50020019000906C48006848
:1003E00040F480306A49086000BF6948006800F442
:1003F000003000900198401C0190009818B90198B5
:10040000B0F5A06FF1D16248006800F4003010B17F
:100410000120009001E0002000900098012843D1C5
:100420005C48006840F010005A49086008460068BF
:1004300020F0030008600846006840F002000860F1
:10044000534840685249486008464068486008463A
:10045000406840F4806048600846406820F47C10A2
:1004600048600846406840F4E81048600846006864
:1004700040F08070086000BF4548006800F00070E0
:100480000028F9D04248406820F003004049486005
:100490000846406840F00200486000BF3C484068A1
:1004A00000F00C000828F9D10CBD10B5FFF792FF41
:1004B00010BD10B53648006840F0010034490860AE
:1004C0000846406834490840314948600846006899
:1004D000324908402E4908600846006820F4802010
:1004E00008600846406820F4FE0048604FF41F0092
:1004F0008860FFF7DAFF4FF000602949086010BDFF
:1005000010B5002100200022214B5B6803F00C0194
:1005100021B1042906D0082928D107E0214B224C1B
:10052000236027E01F4B204C236023E0184B5B68BF
:1005300003F47010164B5B6803F48032022303EB64
:10054000904022B9194B4343174C23600DE0104BE8
:100550005B6803F4003323B1144B4343124C236014
:1005600003E0104B4343104C236003E00D4B0E4C53
:10057000236000BF00BF064B5B68C3F303130C4C42
:10058000E15C094B1B68CB40074C236010BD0000A9
:1005900000100240002002400000FFF8FFFFF6FEBE
:1005A00008ED00E000127A002800002000093D005C
:1005B0002C00002000B589B00121480601F09FFE03
:1005C0000121042001F08EFE4FF40060ADF804001C
:1005D00048208DF8070003208DF8060001A9F9488E
:1005E00001F0C4FB4FF48050ADF8040018208DF8E2
:1005F000070001A9F34801F0B9FBF34800F05EFEE3
:1006000006A800F07FFF00208DF81E008DF81F0067
:100610008DF820008DF821008DF8220001208DF842
:10062000230000208DF81A008DF81B0001208DF8A2
:100630001C0002208DF81D008103E44801F029FC14
:1006400048B14FF48071DF4801F023FC18B13C2021
:10065000ADF818002EE04FF40041DC4801F019FC21
:1006600048B94FF48071D74801F013FC18B130201D
:10067000ADF818001EE04FF40041D44801F009FC29
:1006800048B14FF48071CF4801F003FC18B918202D
:10069000ADF818000EE04FF40041CC4801F0F9FB32
:1006A00040B94FF48071C74801F0F3FB10B90C203A
:1006B000ADF8180006A9C44800F019FE00208DF816
:1006C00012008DF8130001208DF814000020ADF801
:1006D0000800ADF80A00ADF80C00ADF80E00ADF85A
:1006E000100001208DF8150002A800F08AFE0122FA
:1006F0000221B54801F084F914208DF80000012092
:100700008DF8010000208DF8020001208DF8030013
:10071000684600F06AFD09B000BD00B585B0002054
:10072000AB4908606A460021A74801F04EF840F244
:100730001451009888426ED19DF808000028FAD123
:100740009DF80A000128F6D1002240F22551A14867
:1007500002F015FE9DF80B00392871D2DFE800F099
:100760001D23272B2F33373B3F43474B4F53575CBA
:100770006064686C7175797D8185898D9195999D8D
:10078000A1A5A9ADB1B5B9BDC1C5C9CDD1D5D9DD79
:10079000E1E5F0F4F8FCEBEAE90000F0D5FC00201C
:1007A0008D490870E9E001208B490870E5E00220DE
:1007B00089490870E1E0032087490870DDE00420E2
:1007C00085490870D9E0052083490870D5E00620E6
:1007D00081490870D1E007207F490870CDE00820EA
:1007E0007D490870C9E009207B490870C5E00A20EE
:1007F00079490870C1E00B2077490870BDE00C20F2
:1008000075490870B9E00D2073490870B5E00E20F5
:1008100071490870B1E0B1E00F206F490870ACE099
:1008200010206D490870A8E011206B490870A4E001
:10083000122069490870A0E01320674908709CE005
:100840009AE014206449087097E015206249087006
:1008500093E01620604908708FE017205E49087009
:100860008BE018205C49087087E019205A4908700D
:1008700083E01A20584908707FE01B205649087011
:100880007BE01C205449087077E01D205249087015
:1008900073E01E20504908706FE01F204E49087019
:1008A0006BE020204C49087067E021204A4908701D
:1008B00063E02220484908705FE023204649087021
:1008C0005BE024204449087057E025204249087025
:1008D00053E02620404908704FE027203E49087029
:1008E0004BE028203C49087047E029203A4908702D
:1008F00043E02A20384908703FE02B203649087031
:100900003BE02C203449087037E02D203249087034
:1009100033E02E20304908702FE02F202E49087038
:100920002BE030202C49087027E031202A4908703C
:1009300023E01DE018E013E00EE009E004E0FFE72B
:1009400032202549087018E033202349087014E04C
:1009500034202149087010E035201F4908700CE050
:1009600036201D49087008E037201B49087004E054
:1009700038201949087000E000BF00BF05B000BD75
:10098000F0B585B006460F46002440F29440009032
:10099000002001908DF808008DF8090002208DF8E4
:1009A0000A0000BF05E0315D0DF10B000155601C30
:1009B00084B2082CF7DB6946034800F011FE0546B7
:1009C00000240DE00008014000640040000C0140DC
:1009D000B8812142003801403C000020601C84B2F4
:1009E0002946084800F094FE18B140F6FF70844292
:1009F000F4DB40F6FF70844202DB012005B0F0BD5D
:100A00000020FBE70064004008B50121402001F010
:100A100069FC0220ADF8000001208DF8020048209A
:100A20008DF803006946414801F0A0F9012120201A
:100A300001F058FC4FF6FF70ADF8000001208DF872
:100A4000020048208DF803006946394801F08EF90C
:100A50000121102001F046FC4FF47070ADF8000049
:100A600001208DF8020048208DF8030069463148C6
:100A700001F07CF90121042001F034FC4FF4014025
:100A8000ADF8000001208DF8020048208DF8030029
:100A90006946294801F06AF90121082001F022FC89
:100AA0004CF60740ADF8000003208DF80200482006
:100AB0008DF803006946214801F058F9012108200A
:100AC00001F010FC4FF40040ADF8000003208DF859
:100AD000020028208DF803006946184801F046F905
:100AE0000121082001F0FEFB4FF47070ADF800000A
:100AF00003208DF8020048208DF8030069460F4856
:100B000001F034F90221094801F0DDF94FF6FF71D7
:100B1000074801F0D8F94FF47071064801F0D3F995
:100B20004FF40141044801F0CEF908BD001801401E
:100B3000001401400010014000080140000C014079
:100B400008B50121042001F0CDFB4FF4F870ADF899
:100B5000000001208DF8020010208DF80300694686
:100B60000F4801F003F90121082001F0BBFB4FF40D
:100B70004050ADF8000001208DF8020010208DF8E3
:100B800003006946074801F0F1F84FF44051054869
:100B900001F09BF9F021024801F095F908BD000031
:100BA00000080140000C014010B504466FF004003D
:100BB00000F065FBE11704EB5171C1F3C701814AF5
:100BC00011701046007800EB4001C1EBC0104FF6E9
:100BD000FF7101EAC0007C49088010BD01467A4AD5
:100BE00012884A434FF0E0235A6100229A610122A1
:100BF0001A6100BF4FF0E022106900F001021AB143
:100C000000F48032002AF5D000224FF0E0231A6170
:100C10009A61704701466B4A12784A434FF0E023CD
:100C20005A6100229A6101221A6100BF4FF0E0224E
:100C3000106900F001021AB100F48032002AF5D0E8
:100C400000224FF0E0231A619A6170477FB5044695
:100C50000D460121022001F052FB41F28830ADF82F
:100C6000080041F61F40ADF804000020ADF80A006E
:100C7000ADF8060001A9554801F06CFC01224121A4
:100C8000524801F0DEFF1D208DF8000000208DF895
:100C9000010003208DF8020001208DF80300684652
:100CA00000F0A3FA0121494801F0B0FF7FBD10B563
:100CB000474800784749097801EB00104649087019
:100CC000464800784870CC2088706920C87002219E
:100CD0004148FFF755FE10BD10B501213B4802F019
:100CE0005EFA00286CD00121384802F069FA3C48CD
:100CF0000088401C3A4908800988002914DD3849D9
:100D0000088800EBD0714910A0EB410161B930486F
:100D10000078401C2E490870084600780F2801DD35
:100D200000200870FFF7C3FF2E48007890B92E48C6
:100D30000078012807D12D48006808B9012000E09B
:100D400000202A49086028480078B8B900202749BF
:100D5000086013E023480078012808D12348006880
:100D600008B9012000E000202049086006E01D4885
:100D70000078022802D101201C4908601C48007834
:100D800028B11B480078401E1949087002E0012074
:100D90001849086018480078012811D117480088C0
:100DA000401C164908800846008815490988884271
:100DB00006DD0020104908701249087008490880B3
:100DC00010BD00003E000020400000200004004054
:100DD000480000203C000020420000203D00002090
:100DE000460000201900002010000020B0812142A0
:100DF00049000020900121420E0000201600002032
:100E0000140000201800002010B54FF4A06000F07E
:100E1000E7F910BD014600BF704700BFD14A1288F4
:100E200002F04002002AF9D0C2B2CE4B1B1D1A803C
:100E3000704710B586B00446012144F2050001F068
:100E400051FA4FF40070ADF8140003208DF816002D
:100E500018208DF8170005A9C34800F087FF4FF44C
:100E60008060ADF8140004208DF8170005A9BE4875
:100E700000F07CFF25208DF8000003208DF8010094
:100E80008DF8020001208DF80300684600F0ADF9EE
:100E900001940020ADF80800ADF80A00ADF80C0090
:100EA000ADF810000C20ADF80E0001A9AD4802F01D
:100EB000CEF9012240F22551AA4802F060FA012140
:100EC000A84802F050FA06B010BD10B540F2255106
:100ED000A44802F039FB10B3A24802F0B5FAC4B23C
:100EE000A248007800F08000C8B9A048007800F05F
:100EF000400060B10A2C03D000209C49087020E01B
:100F00009A48007840F080009849087019E00D2C4C
:100F100006D19648007840F040009449087010E0EF
:100F20009248007800F03F0091490C548F480078B7
:100F3000401C8E490870084600783F2801DD0020DB
:100F4000087010BD10B586B004460121042001F0E0
:100F5000C9F90121480401F0D2F90420ADF81400C8
:100F600003208DF8160018208DF8170005A97E487B
:100F700000F0FCFE0820ADF8140004208DF81700E6
:100F800005A9794800F0F2FE26208DF80000032024
:100F90008DF801008DF8020001208DF803006846ED
:100FA00000F023F901940020ADF80800ADF80A0024
:100FB000ADF80C00ADF810000C20ADF80E0001A942
:100FC0006C4802F044F901216A4802F0CCF906B0FD
:100FD00010BD6849091D088000BF6649098801F0F5
:100FE00040010029F9D070473EB5044662A207CA05
:100FF0008DE80700002063490860C820FFF7EEFD78
:10100000642094FBF0F03030C0B28DF805000A2067
:1010100094FBF0F00A2190FBF1F201FB120030305A
:10102000C0B28DF806000A2094FBF0F100FB1140DD
:101030003030C0B28DF80700002505E01DF805002E
:10104000FFF7C7FF681CC5B2082DF7DB4FF4C87067
:10105000FFF7C4FD00BF01214B4800F01AFF012833
:10106000F9D00120474908603EBD38B547A0006867
:101070000090002043490860C820FFF7AFFD00241E
:1010800005E01DF80400FFF7A4FF601CC4B2022CA9
:10109000F7DB00BF01213C4800F0FBFE0128F9D03E
:1010A00038BD0CB5024641208DF8000046208DF871
:1010B00001003A208DF802000A2092FBF0F0303057
:1010C000C0B28DF803000A2092FBF0F100FB112062
:1010D0003030C0B28DF80400002305E01DF8030095
:1010E000FFF777FF581CC3B2052BF7DB0CBD70B5BB
:1010F00004460020234908603C2025490870C82088
:10110000FFF76CFD23480078234948710846847135
:1011100020480078C0F1D900001B0872002505E0C6
:101120001D49485DFFF755FF681CC5B20A2DF7DB66
:101130004FF4C870FFF752FD00BF0121124800F0C4
:10114000A8FE0028F9D070BD00B5002205E01349C3
:10115000885CFFF73EFF501CC2B20A2AF7DB00BDD5
:101160007047000000380140000801407000002076
:10117000C00000200044004041373A303030303069
:101180000000000090012142000C014041340000A9
:10119000490000206B0000204C0000205600002079
:1011A0000948804709480047FEE7FEE7FEE7FEE7FB
:1011B000FEE7FEE7FEE7FEE7FEE7FEE70448054937
:1011C000054A064B70470000B3040008ED00000814
:1011D0006001002060070020600300206003002001
:1011E00031490143314A1160704770B50021002335
:1011F0000F22C47804B32D4C246804F4E064C4F5D1
:10120000E064210AC1F10403CA40447804FA03F1FE
:101210008478144021430901254C0678A1550478AF
:1012200004F01F050124AC4005786D11AD0005F1F7
:10123000E025C5F8004109E0047804F01F05012409
:10124000AC401C4D0678761145F8264070BD1A4A10
:101250000A400243154B1B1F1A60704739B1134AED
:10126000121D12680243114B1B1D1A6006E00F4A43
:10127000121D126882430D4B1B1D1A607047042813
:1012800008D14FF0E021096941F004014FF0E0225C
:10129000116107E04FF0E021096921F004014FF0EE
:1012A000E0221161704700000000FA050CED00E03B
:1012B00000E400E080E100E080FFFF1F10B504467D
:1012C000FE48844209D10121480601F032F800218C
:1012D0004FF0007001F02DF808E00121880601F0C0
:1012E00028F800214FF0806001F023F810BD30B5E0
:1012F000024600200023146824F0020414601468DD
:1013000044F00104146000E05B1C546804F0010424
:101310001CB94FF6FF74A342F6D1546804F00104DF
:101320000CB900206CE08C79012C04D1146844F0D5
:101330008004146003E0146824F080041460CC7905
:10134000012C04D1146844F04004146003E01468D4
:1013500024F0400414600C7A012C04D1146844F089
:101360002004146003E0146824F0200414604C7A14
:10137000012C04D1146844F01004146003E01468D4
:1013800024F0100414608C7A012C04D1146844F009
:101390000804146003E0146824F008041460CC7A94
:1013A000012C04D1146844F00404146003E01468B0
:1013B00024F0040414608C78A407CD7844EA056412
:1013C0000D7944EA05444D7944EA05540D886D1EB3
:1013D0002C43D461146824F001041460002300E05D
:1013E0005B1C546804F001041CB14FF6FF74A34267
:1013F000F6D1546804F001040CB1002000E0012093
:1014000030BD10B50021837A012202FA03F1AC4A03
:10141000126842F00102AA4B1A60A94A1C321268F3
:101420008A43A74B1C331A60027BCAB9A44A0C3208
:1014300012688A43A24B0C331A604288C38842EA7E
:1014400003439F4A4032847A42F8343002888388CA
:1014500042EA03439A4A4032847A02EBC402536060
:10146000027B012A19D1964A0C3212680A43944B26
:101470000C331A604288038842EA0343904A4032A0
:10148000847A42F83430C288838842EA03438C4A23
:101490004032847A02EBC4025360C27A3AB9884A75
:1014A000121D12688A43864B1B1D1A6006E0844A8F
:1014B000121D12680A43824B1B1D1A60028932B941
:1014C0007F4A143212688A437D4B14331A600289B2
:1014D000012A06D17A4A143212680A43784B14332F
:1014E0001A60427B012A06D1754A1C3212680A43EF
:1014F000734B1C331A60724A126822F00102704B5F
:101500001A6010BD00218171C17101724172817236
:10151000C1728170C17003210171022141710121E9
:10152000018070476649096841F00101644A116011
:101530001146096843F60E729143614A11601146E3
:10154000096841EA002111601146096821F0010192
:101550001160704721B1026842F48032026003E0FA
:10156000026822F4803202607047E1B1026842F002
:10157000800202604FF4C272125842F480734FF43A
:10158000C27213504FF4CA72125842F480734FF46F
:10159000CA7213504FF4D272125842F480734FF44F
:1015A000D27213501BE0026822F0800202604FF4F6
:1015B000C272125822F480734FF4C27213504FF467
:1015C000CA72125822F480734FF4CA7213504FF447
:1015D000D272125822F480734FF4D27213507047B3
:1015E00010B502460020936803F08063B3F1806F6A
:1015F00000D110E0936803F00063B3F1006F01D1F4
:10160000012008E0936803F08053B3F1805F01D1BB
:10161000022000E00420042879D002F5C07303EB17
:1016200000131B6803F0010402F5C07303EB001301
:101630001C600B7A7BB94B7A0C8843EA445302F561
:10164000C07404EB00142468234302F5C07404EB57
:101650000014236010E00B7A4C6843EAC4034C7A10
:10166000234302F5C07404EB00142468234302F5FD
:10167000C07404EB001423608B7A03F00F038B72A9
:1016800002F5C07303EB00135B6823F00F0402F54F
:10169000C07303EB00135C6002F5C07303EB00132F
:1016A0005B688C7A234302F5C07404EB001463601A
:1016B0008B7B1C064B7B44EA034403E00064004040
:1016C000006600400B7B44EA0323CC7A234302F5F7
:1016D000C07404EB0014A3608B7C1C064B7C44EAB2
:1016E00003440B7C44EA0323CC7B234302F5C07400
:1016F00004EB0014E36002F5C07303EB00131B68F6
:1017000043F0010402F5C07303EB00131C6010BD2D
:1017100010B50246002321B1012907D002290FD1BB
:1017200009E09068F94C00EA04030BE09068F84C7B
:1017300000EA040306E09068F64C00EA040301E0C6
:10174000002300BF00BFF44C181BA34216D007DCD7
:1017500083B16FF08060184470B1022818D111E095
:10176000B0F5007F10D0ED4C204448B1B0F5003FFB
:101770000ED10BE002230DE000230BE0002309E073
:10178000002307E0012305E0012303E0012301E03A
:10179000002300BF00BFD8B210BD21B1012907D07E
:1017A00002290FD109E0826842F0800282600AE0DB
:1017B000826842F40042826005E0826842F40002DE
:1017C000826000E000BF00BF704710B500F5D8731D
:1017D00003EB01131B6803F004031372137A53B96C
:1017E00000F5D87303EB01131B6840F2FF7404EAA1
:1017F0005353136009E000F5D87303EB01131B6822
:101800006FF0604404EAD303536000F5D87303EB30
:1018100001131B6803F00203537200F5D87303EB46
:1018200001135B6803F00F03937200F5D87303EBA9
:1018300001135B681B0AD37400F5D87303EB011323
:101840009B68D37200F5D87303EB01139B681C0AE5
:10185000147300F5D87303EB01139B681C0C5473CD
:1018600000F5D87303EB01139B681B0E937300F50F
:10187000D87303EB0113DB68D37300F5D87303EB64
:101880000113DB681C0A147400F5D87303EB011311
:10189000DB681C0C547400F5D87303EB0113DB6890
:1018A0001B0E937421B9C36843F02003C36003E0A7
:1018B000036943F02003036110BD21B9C26842F0FF
:1018C0002002C26003E0026942F020020261704718
:1018D0000246002019B9D36803F0030006E001298D
:1018E00003D1136903F0030000E00020704710B536
:1018F00002460B4600204FF6FF71BBB9146824F076
:10190000020444F00104146000E0491E546804F02D
:101910000304012C01D00029F7D1546804F003041A
:10192000012C01D0002032E0012030E0012B13D146
:10193000146824F00304146000E0491E546804F0A5
:1019400003040CB10029F8D1546804F003040CB16D
:1019500000201CE001201AE0022B17D1146824F0AB
:10196000010444F00204146000E0491E546804F0CD
:101970000304022C01D00029F7D1546804F00304B9
:10198000022C01D0002002E0012000E0002010BD68
:10199000014600200A6822F0010242F002020A60B9
:1019A0004A6802F00302022A00D101207047014672
:1019B0004FF6FF7200200B6823F002030B6000E07B
:1019C000521E4B6803F00203022B01D1002AF7D10B
:1019D0004B6803F00203022B00D001207047014640
:1019E00000208A6902F070007047014600208A6971
:1019F000100E7047014600208A69C2F30740704705
:101A00001AB143690B43436102E043698B4343616D
:101A1000704710B50246002001F4700343B193698A
:101A2000C1F3130423400BB101202DE000202BE073
:101A300001F0807343B15368C1F3130423400BB129
:101A4000012021E000201FE001F0006343B1936812
:101A5000C1F3130423400BB1012015E0002013E073
:101A600001F0007343B1D368C1F3130423400BB1F9
:101A7000012009E0002007E01369C1F313042340AB
:101A80000BB1012000E0002010BD0022244B994240
:101A900002D10023836111E0C1F3130201F000734E
:101AA0000BB1C2600AE001F080630BB1026105E096
:101AB00001F000630BB1826000E0426070470246B3
:101AC000002002EA01030BB1012000E00020704772
:101AD00070B504460D46002660692840002872D083
:101AE000B5F5807F69D01DDC082D42D006DC012DC4
:101AF0002DD0022D31D0042D7FD134E0102D3ED0D9
:101B0000202D42D0402D78D145E000000300000494
:101B10000003000800000310000100080001FFF7A7
:101B20007000F030B5F5004F61D009DCB5F5007FED
:101B30004AD0B5F5806F4DD0B5F5006F5DD150E05E
:101B4000B5F5803F2DD0B5F5003F56D12FE0A06808
:101B50005549FFF7B4FF064651E0E0680321FFF75F
:101B6000AEFF06464BE0E0680821FFF7A8FF0646F7
:101B700045E0E0681021FFF7A2FF06463FE020693C
:101B80000321FFF79CFF064639E020690821FFF793
:101B900096FF064633E020691021FFF790FF0646C6
:101BA0002DE060680821FFF78AFF064627E060689D
:101BB0001021FFF784FF064621E0A0690121FFF70D
:101BC0007EFF06461BE01BE0A0690221FFF777FFBE
:101BD000064614E0A0690421FFF771FF06460EE0F7
:101BE0000BE0A0697021FFF76AFF064607E0606816
:101BF0000421FFF764FF064601E0002600BF00E075
:101C00000026304670BDB1F5007F3AD00FDC2029A8
:101C100028D006DC01291CD004291DD0082940D178
:101C20001DE0402921D0B1F5807F3AD126E0B1F501
:101C3000004F31D006DCB1F5806F25D0B1F5006FD3
:101C40002FD124E0B1F5803F12D0B1F5003F28D16B
:101C500011E0154A826025E00822C26022E01022CD
:101C6000C2601FE0082202611CE01022026119E03C
:101C70000822426016E01022426013E00422426013
:101C800010E0042242600DE0042242600AE00022DB
:101C900082610422426005E00022826104224260E7
:101CA00000E000BF00BF70470101010010B504460D
:101CB000CC48844208D10121042000F02DFB0021F2
:101CC000042000F029FB46E0C748844208D10121E6
:101CD000082000F021FB0021082000F01DFB3AE065
:101CE000C248844208D10121102000F015FB0021D8
:101CF000102000F011FB2EE0BD48844208D10121E4
:101D0000202000F009FB0021202000F005FB22E04C
:101D1000B848844208D10121402000F0FDFA00219A
:101D2000402000F0F9FA16E0B348844208D10121BE
:101D3000802000F0F1FA0021802000F0EDFA0AE0A6
:101D4000AE48844207D10121801500F0E5FA002158
:101D5000A01500F0E1FA10BD10B50121084600F011
:101D6000DBFA0021012000F0D7FA10BD2DE9F04187
:101D7000024600250026002000230024002791F8B9
:101D800003C00CF00F0591F803C00CF0100CBCF16F
:101D9000000F03D091F802C04CEA050591F800C08D
:101DA000BCF1000F31D0146800202BE04FF0010C83
:101DB0000CFA00F3B1F800C00CEA03069E4220D1F1
:101DC00083004FF00F0C0CFA03F7BC4305FA03FC39
:101DD0004CEA040491F803C0BCF1280F06D14FF07F
:101DE000010C0CFA00FCC2F814C00AE091F803C020
:101DF000BCF1480F05D14FF0010C0CFA00FCC2F801
:101E000010C0401C0828D1D31460B1F800C0BCF148
:101E1000FF0F34DD546800202EE000F1080C4FF075
:101E2000010808FA0CF3B1F800C00CEA03069E4260
:101E300021D183004FF00F0C0CFA03F7BC4305FAD5
:101E400003FC4CEA040491F803C0BCF1280F05D14F
:101E500000F1080C08FA0CF8C2F8148091F803C0DD
:101E6000BCF1480F07D100F1080C4FF0010808FA47
:101E70000CF8C2F81080401C0828CED35460BDE88E
:101E8000F0814FF6FF710180022181700421C17041
:101E900070470246002093680B400BB1012000E020
:101EA000002070470146886880B2704702460020D3
:101EB000D3680B400BB1012000E0002070470146C1
:101EC000C86880B2704701617047416170470AB1CC
:101ED000016100E041617047C16070474FF480329A
:101EE0000A43826181618261826982697047024628
:101EF0000020434B18684FF68073184040EA0210E8
:101F000008433F4B186070473E49C8617047F0B5C1
:101F10000A46002300240021002500F00046B6F107
:101F2000004F02D1364EF16901E0354E7168C0F3C1
:101F3000034583B200F44016B6F5401F08D121F0E6
:101F400070612F4E766826F070662D4F7E6012E02D
:101F500000F48016B6F5801F06D1032606FA05F4B4
:101F6000A14341F0706106E0460D360103FA06F622
:101F7000B14341F0706122B1460D360103FA06F615
:101F8000314300F00046B6F1004F02D11C4EF16122
:101F900001E01B4E7160F0BD30B500228B071C0FB5
:101FA0000F2303FA04F2164B08338C1053F8243035
:101FB0009343134C08348D1044F8253023468C107D
:101FC00053F824308C07240F00FA04F423430C4CFC
:101FD00008348D1044F8253030BD0A49DC310860E2
:101FE0007047000000080140000C01400010014053
:101FF0000014014000180140001C01400020014075
:102000000000014000002042DF48006840F001006D
:10201000DD49086008464068DC490840DA49486004
:1020200008460068DA490840D74908600846006851
:1020300020F4802008600846406820F4FE004860D4
:102040004FF41F0088607047CF49096821F4803140
:10205000CD4A11601146096821F480211160B0F564
:10206000803F03D0B0F5802F0ED106E0C649096845
:1020700041F48031C44A116007E0C349096841F462
:10208000A021C14A116000E000BF00BF704710B539
:1020900001460022002300204A11012A02D1BA4C35
:1020A000236806E0022A02D1B74C236A01E0B64C4D
:1020B000636A01F01F02012494401C400CB101200E
:1020C00000E0002010BD38B500200090002400255D
:1020D00000BF3120FFF7DBFF05460098401C009051
:1020E0000098B0F5A06F01D0002DF2D03120FFF79D
:1020F000CEFF08B1012400E00024204638BD01468F
:102100000020A14A106820F0F80040EAC1001060E9
:102110007047A04908607047024600209A4B5868F3
:1021200020F47C1042EA01031843974B5860704733
:1021300098490866704701460020934A506820F08D
:1021400003000843506070478F48406800F00C005F
:102150007047014600208C4A506820F0F000084388
:102160005060704701460020874A506820F4E060C4
:1021700008435060704701460020834A506820F4AD
:10218000605040EAC1005060704729B17E4A527ADF
:1021900002437D4B5A7204E07B4A527A82437A4B67
:1021A0005A7270477B49D831086070470146002059
:1021B000754A506820F44040084350607047002141
:1021C000714A20321170704A82F82010012802D022
:1021D00004280AD104E001216B4A2032117005E085
:1021E0000521694A2032117000E000BF00BF70472E
:1021F0006949086070476449096A0143624A11628B
:102200007047654944390860704730B500210022A5
:10221000002400235C4D6D6805F00C0121B10429F8
:1022200005D0082923D105E05C4D056022E05B4D17
:1022300005601FE0544D6D6805F47012524D6D68D5
:1022400005F48034022505EB92421CB9544D5543E8
:1022500005600BE04C4D6D6805F400351DB1504D27
:102260005543056002E04D4D5543056002E04B4D7E
:10227000056000BF00BF444D6D6805F0F00109091D
:10228000484D6B5C0568DD4045603F4D6D6805F469
:10229000E061090A434D6B5C4568DD4085603A4D5D
:1022A0006D6805F46051C90A3E4D6B5C4568DD40C0
:1022B000C560354D6D6805F44041890B3A4D6B5C46
:1022C000C568B5FBF3F5056130BD29B12E4A5269E9
:1022D00002432D4B5A6104E02B4A526982432A4B38
:1022E0005A61704729B1284A92690243264B9A6184
:1022F00004E0254A92698243234B9A61704729B1D1
:10230000214AD2690243204BDA6104E01E4AD269B5
:1023100082431D4BDA61704729B11B4AD2680243E0
:10232000194BDA6004E0184AD2688243164BDA602F
:10233000704729B1144A12690243134B1A6104E031
:10234000114A12698243104B1A6170471249403991
:10235000086070470F49C86470470B49C8717047DF
:102360000948406A40F0807007494862704701465A
:102370000020054A92680A400AB1012000E00020CE
:102380007047014988727047001002400000FFF852
:10239000FFFFF6FE000042428004424200127A0033
:1023A00000093D00710000208100002010B50446A6
:1023B000FE48844208D10121C014FFF7ADFF00217F
:1023C000E014FFF7A9FFC4E0B4F1804F08D1012168
:1023D0000846FFF7AEFF00210120FFF7AAFFB8E093
:1023E000F348844208D101210220FFF7A2FF002117
:1023F0000220FFF79EFFACE0EE48844208D10121A5
:102400000420FFF796FF00210420FFF792FFA0E0D1
:10241000E948844208D101210820FFF78AFF002102
:102420000820FFF786FF94E0E448844208D10121A8
:102430001020FFF77EFF00211020FFF77AFF88E0D1
:10244000DF48844208D101212020FFF772FF0021DC
:102450002020FFF76EFF7CE0DA48844208D101219A
:102460004014FFF759FF00216014FFF755FF70E09B
:10247000D548844209D10121C804FFF74DFF00214E
:102480004FF40020FFF748FF63E0D048844209D1B1
:1024900001210805FFF740FF00214FF48010FFF7EE
:1024A0003BFF56E0CA48844209D101214805FFF7A5
:1024B00033FF00214FF40010FFF72EFF49E0C5481D
:1024C000844208D101214020FFF733FF0021402042
:1024D000FFF72FFF3DE0C048844208D10121802052
:1024E000FFF727FF00218020FFF723FF31E0BB48E3
:1024F000844208D101218015FFF71BFF0021A015A0
:10250000FFF717FF25E0B648844209D101210804EE
:10251000FFF702FF00214FF48030FFF7FDFE18E0C7
:10252000B048844209D101214804FFF7F5FE00219B
:102530004FF40030FFF7F0FE0BE0AB48844208D1C7
:1025400001218804FFF7E8FE00214FF48020FFF707
:10255000E3FE10BD00220288944B98420ED0994BA6
:1025600098420BD0B0F1804F08D0914B984205D0E3
:10257000904B984202D0904B984204D14FF68F7303
:102580001A404B881A438D4B984207D08C4B984287
:1025900004D04FF6FF431A40CB881A4302808B8841
:1025A00083850B880385814B98420BD0854B9842DD
:1025B00008D08B4B984205D08A4B984202D08A4B68
:1025C000984201D10B7A038601238382704770B54C
:1025D000002400220023058C4FF6FE76354005844A
:1025E000028C8388048B4FF68F752C40B51E2C40CF
:1025F0000D882C43751E2A400D892A434D882A4395
:102600006A4DA8420BD06F4DA84208D0744DA84225
:1026100005D0744DA84202D0734DA84213D14FF695
:10262000F7752A404D892A434FF6FB752A408D885D
:102630002A434FF6FF652B404FF6FF552B408D89FF
:102640002B43CD892B4383800483CD8885860284E8
:1026500070BD70B5002400220023058C4FF6EF7684
:1026600035400584028C8388048B48F6FF752C4026
:102670004FF6FF452C400D884FF6FF7606EA0525FC
:102680002C434FF6DF752A400D8906EA05152A43CB
:102690004D8806EA05152A43444DA84202D0494D0B
:1026A000A8421DD14FF67F752A404D894FF6FF761F
:1026B00006EA05152A434FF6BF752A408D8806EABB
:1026C00005152A434FF6FF352B404FF2FF752B407F
:1026D0008D8906EA85052B43CD8906EA85052B43BE
:1026E00083800483CD880587028470BD70B5002483
:1026F00000220023058C4FF6FF6635400584028CCE
:102700008388848B4FF68F752C404FF6FC752C40D8
:102710000D882C434FF6FF552A400D894FF6FF7662
:1027200006EA05252A434D8806EA05252A431F4D5A
:10273000A84202D0234DA8421DD14FF2FF752A4076
:102740004D894FF6FF7606EA05252A434FF6FF35F9
:102750002A408D8806EA05252A434EF6FF752B4050
:102760004DF6FF752B408D8906EA05152B43CD8963
:1027700006EA05152B4383808483CD8885870284F0
:1027800070BD70B5002200230024058C4EF6FF7644
:1027900035400584038C8488828B48F6FF752A4077
:1027A0004FF6FF452A400D8820E00000002C014034
:1027B0000004004000080040000C004000100040F1
:1027C0000014004000340140004C01400050014022
:1027D0000054014000180040001C00400020004050
:1027E0000040014000440140004801404FF6FF76A0
:1027F00006EA05252A434DF6FF752B400D8906EAAA
:1028000005352B434D8806EA05352B43FA4DA84282
:1028100002D0FA4DA84208D14BF6FF752C408D89A5
:102820004FF6FF7606EA85152C4384808283CD8897
:10283000A0F84050038470BD828B4FF2FF331A40E2
:102840008283828B4FF6FF7303EA01231A4382834C
:102850007047F0B50C461546002200210026078C73
:102860004EF6FF7C07EA0C070784828B018C4FF63B
:10287000FF7707EA043640F6FF473A404FF6FF7706
:1028800007EA05273A434FF6FF7707EA03373A434B
:10289000D94FB8420ED0D94FB8420BD0B0F1804FCB
:1028A00008D0D74FB84205D0D64FB84202D0D64F45
:1028B000B84206D14DF6FF77394046F48057394388
:1028C00005E047F6FF57394044F480573943828387
:1028D0000184F0BD828B4FF6F3731A408283828BA2
:1028E0000A4382837047F0B50C461546002200214A
:1028F0000026078C4FF6FF6C07EA0C070784828BD3
:10290000018C4FF6FF7707EA04264FF60C773A4022
:102910004FF6FF7707EA03172F433A43B64FB84203
:102920000ED0B64FB8420BD0B0F1804F08D0B44FA4
:10293000B84205D0B34FB84202D0B34FB84206D127
:102940004FF6FF57394046F48077394305E04FF2A0
:10295000FF57394044F48077394382830184F0BDC6
:10296000028B4FF2FF331A400283028B4FF6FF7344
:1029700003EA01231A4302837047F0B50C4615465B
:10298000002200210026078C4FF6EF7C07EA0C0797
:102990000784028B018C4FF6FF7707EA041640F696
:1029A000FF473A404FF6FF7707EA03373A434FF6BF
:1029B000FF7707EA05273A438F4FB8420ED08F4F73
:1029C000B8420BD0B0F1804F08D08D4FB84205D03F
:1029D0008C4FB84202D08C4FB84206D14FF6DF7709
:1029E000394046F01007394305E04FF65F7739402C
:1029F00044F01007394302830184F0BD028B4FF687
:102A0000F3731A400283028B0A4302837047F0B5C6
:102A10000C46154600220021068C4FF6FE773E40FC
:102A20000684028B018C4FF60C7632407E1C06EA3F
:102A300003162E433243704EB0420ED06F4EB0425A
:102A40000BD0B0F1804F08D06D4EB04205D06D4E26
:102A5000B04202D06C4EB04206D14FF6FD76314006
:102A600044F00106314305E04FF6F576314044F07D
:102A70000106314302830184F0BD70B505460C4662
:102A80005D4885420ED05D4885420BD0B5F1804F40
:102A900008D05B48854205D05A48854202D05A4842
:102AA000854200D100E000BF208850B92389A28868
:102AB00061882846FFF7ABFFE1882846FFF79EFFB5
:102AC00025E0208804280AD12389A2886188284625
:102AD000FFF753FFE1882846FFF742FF17E0208801
:102AE00008280AD12389A28861882846FFF7FBFEBF
:102AF000E1882846FFF7EEFE09E02389A288618875
:102B00002846FFF7A6FEE1882846FFF795FE70BD30
:102B10002DE9F04105460C4600260127608808B9DA
:102B2000022600E00026A088012801D1022700E04B
:102B300001272088A0B92389A28861882846FFF749
:102B400066FFE1882846FFF759FF23893A46314658
:102B50002846FFF712FFE1882846FFF701FF13E040
:102B60002389A28861882846FFF707FFE188284665
:102B7000FFF7F6FE23893A4631462846FFF747FF1E
:102B8000E1882846FFF73AFFBDE8F0810A884B88C4
:102B90001A438B881A43CB881A430B891A434B89F3
:102BA0001A438B891A43A0F8442070474FF6FF71EF
:102BB000818000210180C180418001727047002125
:102BC000018041808180C180018141818181C181F9
:102BD0007047002101804180012181800021C18056
:102BE000018170470021018041808180C180018185
:102BF0004181818170470000002C01400034014078
:102C00000004004000080040000C004021B1028890
:102C100042F00102028004E002884FF6FE731A407F
:102C20000280704731B1B0F8442042F40042A0F86D
:102C3000442005E0B0F84420C2F30E02A0F844207E
:102C400070471AB183890B43838102E083898B43E8
:102C5000838170478182704741EA0203A0F84830BF
:102C600070471AB183890B43838102E083898B43C8
:102C70008381704701894FF6F872114001817047D6
:102C80000A46002101894FF68F73194011430181D3
:102C9000704730B504460D4629462046FFF7F0FF41
:102CA000208940F00700208130BD2DE9F041044625
:102CB0000D4616461F46602D06D13B460122314681
:102CC0002046FFF75AFE05E03B46012231462046EA
:102CD000FFF79DFE29462046FFF7D2FF208940F0EE
:102CE00007002081BDE8F08130B50C460021018944
:102CF000C9B24FF6FF7505EA03251543254329435D
:102D0000018130BD2DE9F04105460E461746984633
:102D1000002443463A4631462846FFF7E5FF2C8912
:102D20004FF6F870044044F007044FF68F700440EB
:102D300044F070042C81BDE8F081F0B504460D46E6
:102D400016461F463B46324629462046FFF7CCFF33
:102D5000208940F480402081F0BD01858282704747
:102D60000A46002101884FF68F73194011430180F4
:102D70007047F0B50C4615461E4600210022002380
:102D80000189028B038C4FF6F877394021434FF6C7
:102D9000FC473A4040F201173A434FF6DD773B409B
:102DA0004FF6FF7707EA06172F433B430181028363
:102DB0000384F0BD0A460021018B4FF68F73194042
:102DC0001143018370470A460021018B48F6FF73C7
:102DD00019404FF6FF7303EA02231943018370473A
:102DE0000A460021818B4FF68F731940114381836E
:102DF00070470A460021818B48F6FF7319404FF651
:102E0000FF7303EA022319438183704721B10288CB
:102E100042F08002028004E002884FF67F731A407D
:102E20000280704721B1828842F00402828004E06F
:102E300082884FF6FB731A408280704721B18288E6
:102E400042F00802828004E082884FF6F7731A404D
:102E50008280704721B1828842F00102828004E0C2
:102E600082884FF6FE731A40828070470A4600211E
:102E7000018B4FF6F77319401143018370470A46DF
:102E80000021018B4FF2FF7319404FF6FF7303EAE5
:102E900002231943018370470A460021818B4FF6B4
:102EA000F77319401143818370470A460021818BD3
:102EB0004FF2FF7319404FF6FF7303EA02231943E1
:102EC000818370470A460021018B4FF6FB7319403E
:102ED0001143018370470A460021018B4FF6FF33EF
:102EE00019404FF6FF7303EA022319430183704729
:102EF0000A460021818B4FF6FB73194011438183F1
:102F000070470A460021818B4FF6FF3319404FF678
:102F1000FF7303EA02231943818370470A460021A5
:102F2000018B4FF67F7319401143018370470A46A6
:102F30000021018BC1F30E014FF6FF7303EA022358
:102F40001943018370470A460021818B4FF67F7336
:102F500019401143818370470A460021818BC1F3D8
:102F60000E014FF6FF7303EA022319438183704772
:102F70000A460021018C4FF6FD731940114301846C
:102F800070470A460021018C4FF6F7731940114330
:102F9000018470470A460021018C4FF6DF73194007
:102FA0004FF6FF7303EA02131943018470470A4680
:102FB0000021018C4FF67F7319404FF6FF7303EA2F
:102FC00002131943018470470A460021018C4FF611
:102FD000FF5319404FF6FF7303EA0223194301849C
:102FE00070470A460021018C4FF2FF7319404FF6DB
:102FF000FF7303EA02231943018470470A46002144
:10300000018C4DF6FF7319404FF6FF7303EA02334C
:1030100019430184704730B5002301248C40A3B2CA
:10302000048C9C430484048C02FA01F5ADB22C4359
:10303000048430BD30B5002304248C40A3B2048C3A
:103040009C430484048C02FA01F5ADB22C43048441
:1030500030BD70B503460020002418461830012505
:103060008D40ACB21D8CA5431D8409B1082909D13E
:1030700000EB6100056825F07005056005681543E3
:1030800005600EE00D1FC5F34E052844056825F4C4
:10309000E045056005684FF6FF7606EA02263543EF
:1030A000056070BD21B1028842F00202028004E096
:1030B00002884FF6FD731A400280704721B10288E2
:1030C00042F00402028004E002884FF6FB731A40CB
:1030D0000280704721B1828842F08002828004E041
:1030E00082884FF67F731A408280704702884FF6BD
:1030F000F7731A40028002880A4302807047828870
:103100004FF68F731A40828082880A43828070470C
:1031100002894FF6F8731A40028102890A4302813C
:10312000704702894FF67F731A40028102890A4371
:10313000028170478184704781857047818670471E
:103140000187704781877047A0F840107047028858
:103150004FF6FF431A40028002880A4302807047FC
:103160000146888E70470146088F70470146888F58
:1031700070470146B1F8400070470146888C70479F
:103180000146088D704702460020138A0B400BB1A0
:10319000012000E000207047CA430282704730B52A
:1031A0000246002000230024158A05EA01039589C0
:1031B00005EA010413B10CB1012000E0002030BD8C
:1031C000CA4302827047000010B50446FB4884429F
:1031D00009D101218803FFF79FF800214FF48040B7
:1031E000FFF79AF832E0F648844209D101214804F9
:1031F000FFF79FF800214FF40030FFF79AF825E021
:10320000F048844209D101218804FFF792F8002197
:103210004FF48020FFF78DF818E0EB48844209D185
:103220000121C804FFF785F800214FF40020FFF7C3
:1032300080F80BE0E548844208D101210805FFF73A
:1032400078F800214FF48010FFF773F810BD2DE9D6
:10325000F04786B005460E460024A24600BFA146B0
:103260000027B08900B100BF2F462C8A4CF6FF70B2
:103270000440F08804432C82AC894EF6F3100440DD
:10328000B08831890843718908430443AC81AC8A12
:103290004FF6FF400440B0890443AC8201A8FEF71A
:1032A000B4FFC648874202D1DDF810A001E0DDF886
:1032B0000CA0A88900F4004040B10AEBCA0000EB62
:1032C0000A1031684900B0FBF1F807E00AEBCA00C8
:1032D00000EB0A1031688900B0FBF1F86420B8FBFC
:1032E000F0F004012009642101FB1089A88900F491
:1032F000004040B1322000EBC900B0FBF1F000F01B
:103300000700044308E0322000EB09106421B0FB01
:10331000F1F000F00F0004432C8106B0BDE8F08707
:103320004FF41651016000218180C18001810C2180
:10333000418100218181704710B502460020108A2A
:103340004FF2FF0318400B884C8823438C8823439B
:10335000CC8823431843108210BD00210180418096
:103360008180C180704721B1828942F400528281FC
:1033700004E082894DF6FF731A4082817047F0B5F0
:103380000346002400260025002040F66A17B942B3
:1033900000D100BF1846C1F3421401F01F060127F7
:1033A00007FA06F5012C01D10C3004E0022C01D102
:1033B000103000E014301AB107682F43076002E0B4
:1033C0000768AF430760F0BD1AB1838A0B4383825D
:1033D00002E0838A8B4383827047028A4FF6F07340
:1033E0001A400282028A0A430282704782894FF29F
:1033F000FF731A40828182890A438281704721B11A
:10340000828942F00202828104E082894FF6FD73D4
:103410001A4082817047028A4FF6DF731A40028297
:10342000028A0A430282704721B1028A42F4804232
:10343000028204E0028A4BF6FF731A400282704750
:10344000C1F308028280704701468888C0F30800F3
:103450007047818941F0010181817047028BD2B2AE
:103460000283028B42EA012202837047028B02F43C
:103470007F420283028B0A430283704721B1828A12
:1034800042F02002828204E0828A4FF6DF731A4003
:103490008282704721B1828A42F01002828204E067
:1034A000828A4FF6EF731A408282704721B1828A76
:1034B00042F00802828204E0828A4FF6F7731A40D3
:1034C0008282704721B1828942F40042828103E006
:1034D0008289C2F30E028281704721B1828A42F44E
:1034E0000062828204E0828A4FF2FF731A40828275
:1034F0007047828A4FF6FB731A408282828A0A439F
:103500008282704721B1828A42F00202828204E004
:10351000828A4FF6FD731A4082827047024600206D
:10352000B1F5007F00D100BF13880B400BB1012023
:1035300000E00020704701F40072B2F5007F00D176
:1035400000BFCA430280704770B5024600240023C2
:103550000025002040F66A16B14200D100BFC1F339
:10356000421501F01F03012606FA03F3012D02D1D3
:103570009689334006E0022D02D1168A334001E0DD
:10358000968A33400C12012606FA04F41688344059
:1035900013B10CB1012000E0002070BD10B5002275
:1035A000002340F66A14A14200D100BF0A12012490
:1035B0009440A3B2DC43048010BD000000380140F9
:1035C0000044004000480040004C004000500040D3
:1035D00070477047704770477047754600F02CF889
:1035E000AE4605006946534620F00700854618B0F0
:1035F00020B5FDF7E3FDBDE820404FF000064FF099
:1036000000074FF000084FF0000B21F00701AC4617
:10361000ACE8C009ACE8C009ACE8C009ACE8C00936
:103620008D46704710B50446AFF300802046BDE8D4
:103630001040FCF7A2BD00000048704700010020C8
:103640006036000800000020880000002801000803
:10365000E836000888000020D80600004401000871
:103660000000000000000000000000000000000159
:1036700000000000780000000000010203040503C0
:10368000010203040506000000A24A040000000035
:103690000000000001020304060708090001000001
:1036A0000000000102030000000000007EFF06226F
:1036B000001E01FEBAEF7EFF0616000000FEE5EFD9
:1036C0007EFF0642000000FEB9EF000A0000000085
:1036D00000000000000102030401020304060708C1
:0836E0000902040608000000C5
:04000005080000ED02
:00000001FF
